:1000000013C01AC019C018C017C016C015C014C03C
:1000100013C012C011C010C00FC00EC00DC03F06EB
:100020005B4F666D7D077F6F11241FBECFE5D1E06A
:10003000DEBFCDBFEAD106C4E3CFF894C09AC29A1E
:100040008DE08A95F1F70000C0988DE08A95F1F770
:100050000000C29878940895F894C298C0988DE0F2
:100060008A95F1F70000C29A8DE08A95F1F70000B9
:10007000C09A78940895F8942DE02A95F1F700003D
:1000800098E00DC0C09886952DE02A95F1F7000004
:10009000C29A2DE02A95F1F70000915049F0C298DC
:1000A0002DE02A95F1F7000080FFECCFC09AEBCF4E
:1000B000B898C298C09A8DE08A95F1F7000086B38F
:1000C000C29A9DE09A95F1F70000C2982DE02A951A
:1000D000F1F70000B89A7894809581700895CF93D5
:1000E000C82FABDF8C2FC7DFB7DFCF91089597B351
:1000F000A1E0B0E0FD0102C0EE0FFF1F8A95E2F71C
:1001000002C0AA0FBB1F6A95E2F7EA2B9E2B97BB92
:1001100088B3E095E823E8BB842F8068822BDFDF7B
:100120000895CF93DF93C82FD62F80E4D8DF85DFE3
:100130008D2F806CA0DF8C2F9EDF8EDFDF91CF9123
:10014000089562E080E4EDDF61E080E4EADF60E0F2
:1001500080E4E7DF0895BF92CF92DF92EF92FF92A3
:100160000F931F93CF93DF938C01EC01083E83E044
:10017000180714F0C7EED3E0112354F00F2EF3E06C
:10018000DF2EF02D0F2EFAE0EF2EF12CF02D17C000
:10019000D195C195D10960E080E4C3DFEFCFDA9457
:1001A000CE01B7013CD3B62EC72E825E9F4FFC0115
:1001B00084916D2DB6DFCB2DDC2DDD2029F01123B0
:1001C00074F7E1E0DE12EBCFDF91CF911F910F9139
:1001D000FF90EF90DF90CF90BF900895992384F027
:1001E00021E08A30910554F021E0EAE0F0E0BF011F
:1001F00016D3CB012F5F6A307105CCF7822F08959B
:10020000919581959109ECCF7F928F929F92AF92B9
:10021000BF92CF92DF92EF92FF920F931F93CF93F3
:10022000DF9300D01F92CDB7DEB7F62E942EE22ECC
:1002300099230CF44DC021E0E11001C020E06C01D5
:10024000883E934034F00F2EF7EECF2EF3E0DF2EF2
:10025000F02DE11008C0C601C1DFB82E52E08513B1
:100260004CC010E04BC0E22E3FC00B2D63C0682D88
:1002700080E457DF81E0800F1E2D96C0E3E0BE12C0
:10028000A2C0E11081C0A1107FC065C0882DE1101F
:10029000AAC0892DA8C0872D023009F080C074C083
:1002A000EF2DF0E0E25EFF4F8491612F3ADF0F9077
:1002B0000F900F90DF91CF911F910F91FF90EF90D2
:1002C000DF90CF90BF90AF909F908F907F900895D8
:1002D0006C01883E934034F00F2EF7EECF2EF3E002
:1002E000DF2EF02DEE24E394D194C194D108C60101
:1002F00075DFB82E52E011E0851310E02AE030E0FF
:10030000C601B9018CD28B83CB01B90188D28A8313
:10031000C60164E670E083D2CB01B90180D2A82E79
:10032000898381E0B81609F4A0CF03E00B190330EC
:1003300008F0B6CF82E090E06C01C918D1087E2C9D
:100340006894992497F8812C33C01C151D0409F476
:1003500095CFA11015C0202F30E0E1E0F0E0EC0FC8
:10036000FD1FE20FF31F808181110AC042E050E0BF
:100370004C0F5D1F240F351FF901908191110FC0A3
:10038000F1E0BF1609F487CFE1E0F0E0EC0FFD1FCC
:10039000E00FF11DE081F0E0E25EFF4F8491612FFC
:1003A000C0DE81E0800F1F5F0F5F833008F078CFE1
:1003B000EE2059F2112309F45ACF1C151D0421F720
:1003C00083E0B81609F3E1E0F0E0EC0FFD1FE00F69
:1003D000F11DE081F0E0E25EFF4FE491F2E0892D53
:1003E000BF1609F453CF8E2BDACF56D1882351F0A4
:1003F000813011F081E00895C39A81E090E0ABDE96
:1004000081E00895C39880E00895CF93DF93CDB73E
:10041000DEB766970FB6F894DEBF0FBECDBFBB9AAE
:10042000C398A89588E198E20FB6F894A89581BD85
:100430000FBE91BD6BE0CE010196F3D028E042E003
:1004400062E080E054DE7DDE2FEF80E792E0215015
:1004500080409040E1F700C0000004E610E00DC0CD
:10046000CE01019633D18B899C89B801C4D12D89E5
:1004700041E089899A89C8DEA895CE010196B5DF49
:10048000882371F32FE788E391E02150804090406A
:10049000E1F700C00000A895F0CFF894BC9A8FEB6C
:1004A00093E00197F1F700C00000BC989AEB9A9591
:1004B000F1F700C086B3E3E3F3E03197F1F700C052
:1004C000000078948295817091E08927089598E0E2
:1004D0000DC0BC9A20EA2A95F1F7BC982AE12A952A
:1004E000F1F700C078948695915069F0F89480FFF8
:1004F000F0CFBC9A20E12A95F1F7BC982AEA2A9518
:10050000F1F700C0EFCF089598E080E007C022E93E
:100510002A95F1F700C07894915071F0F89486957F
:10052000BC9A20E12A95F1F7BC9828E12A95F1F7C9
:10053000B49BEDCF8068EBCF0895AFDF811101C090
:1005400008958CECC4DF81E0FBCF0F931F93CF9312
:10055000DF938C01A2DF811105C0DF91CF911F9144
:100560000F91089583E3B3DFE801085F1F4FCCDFED
:100570008993C017D107D9F781E0EFCFFC01680F4D
:10058000791F80E02CE80BC08695915029F080FF00
:10059000FBCF86958227F9CFE617F70721F09191D7
:1005A000892798E0F4CF0895EF92FF920F931F935D
:1005B000CF93DF937C01C1DF8EEB89DFE7018701F9
:1005C000085F1F4FA1DF8993C017D107D9F768E0F3
:1005D00070E0C701D3DFC82F97DF91E0C81390E028
:1005E000892FDF91CF911F910F91FF90EF90089588
:1005F00054DF811101C00895A0DF88E468DF81E045
:10060000FACFCF93DF93EC0198DF8EE460DF88812F
:100610005EDF89815CDF8A815ADFEADFDF91CF917B
:100620000895FF920F931F93CF93DF9300D01F92F3
:10063000CDB7DEB78C01F62EB7DFF8018281898352
:1006400083818A83FAE0FF16B9F08BE0F81689F00F
:10065000E9E0FE16A1F08FE78B83CE010196D1DF92
:100660000F900F900F90DF91CF911F910F91FF90FE
:1006700008958FE58B83F1CF8FE38B83EECF8FE1EE
:100680008B83EBCF0ADF811101C008958CEC1FDF53
:1006900084E41DDF81E0F9CFCF93DF93EC01FDDE31
:1006A000811104C081E0DF91CF910895CE010896B9
:1006B0004CDF8885883211F082E0F5CFCE0174DFFF
:1006C000882311F080E0EFCF83E0EDCFCF93DF936D
:1006D000EC01D8DF882309F45EC02C81822F90E0E2
:1006E0008095909580769927892B09F057C02FE740
:1006F0003FE482E1215030408040E1F700C000003B
:10070000CE0152DF882309F46BC01D8A898190E0F5
:100710004881242F382F33230CF465C03595279555
:10072000359527953595279535952795398B288BC0
:1007300080959095887F9927892B09F057C081E093
:100740008C8B4195488388818F70282F30E0C901B8
:10075000880F991F82959295907F9827807F982780
:10076000821B930B880F991F880F991F820F931F6D
:10077000880F991F880F991F880F991F9C01992333
:10078000BCF1359527953595279535952795359560
:1007900027953B8B2A8BDF91CF91089526FF0AC0C6
:1007A0009FEB27E239E0915020403040E1F700C054
:1007B0000000A6CF25FF0AC08FEF96E924E0815004
:1007C00090402040E1F700C000009ACF3FE78BE463
:1007D00092E0315080409040E1F700C0000090CF9F
:1007E00081E08D8BD8CF215F3F4F98CF1C8AABCF54
:1007F000215F3F4FC6CFAA1BBB1B51E107C0AA1FF9
:10080000BB1FA617B70710F0A61BB70B881F991FB1
:100810005A95A9F780959095BC01CD01089597FB55
:10082000072E16F4009406D077FD08D0E4DF07FC0D
:1008300005D03EF4909581959F4F089570956195F0
:080840007F4F0895F894FFCFEB
:00000001FF
